:020000040800F2
:10000000D82100204D0100080D100008BD0800088F
:10001000B10F0008DF0200082124000800000000E2
:10002000000000000000000000000000F1120008C5
:10003000FB0500080000000063010008911500089E
:1000400067010008670100086701000867010008F0
:1000500067010008670100086701000867010008E0
:1000600067010008670100086701000867010008D0
:100070004304000867010008450400086701000800
:1000800067010008670100086701000867010008B0
:1000900067010008670100086701000867010008A0
:1000A0006701000867010008670100086701000890
:1000B0006701000867010008670100086701000880
:1000C0006701000867010008670100086701000870
:1000D00067010008A91F0008670100086701000800
:1000E0006701000867010008670100086701000850
:1000F0006701000867010008670100086701000840
:10010000670100086701000867010008670100082F
:10011000670100086701000867010008670100081F
:10012000670100086701000867010008670100080F
:10013000DFF80CD000F0A2F800480047092C0008B6
:10014000D821002080F308887047000006488047C7
:1001500006480047FEE7FEE7FEE7FEE7FEE7FEE7AC
:10016000FEE7FEE7FEE7FEE7411600083101000862
:1001700040EA01039B0703D009E008C9121F08C029
:10018000042AFAD203E011F8013B00F8013B521EA9
:10019000F9D27047D2B201E000F8012B491EFBD220
:1001A00070470022F6E710B513460A460446194682
:1001B000FFF7F0FF204610BD421E12F8013F002B52
:1001C000FBD111F8013B02F8013B002BF9D170473C
:1001D00010B5002200E0521C835C8C5CA34201D16C
:1001E000002BF8D1D8B2E1B2401A10BD30B50446A8
:1001F0000020034600E05B1C934203D2E05CCD5C30
:10020000401BF8D030BD034611F8012B00F8012B3C
:10021000002AF9D1184670472DE9F05F0546002005
:1002200092469B4688460646814640241BE0284667
:1002300041464746224600F042F853465A46C01A05
:10024000914110D311461846224600F029F82D1A84
:1002500067EB01084F4622460120002100F020F8FC
:1002600017EB00094E41201EA4F10104DFDC4846D3
:1002700031462A464346BDE8F09F0000064C074D34
:1002800006E0E06840F0010394E807009847103466
:10029000AC42F6D3FFF750FF0C3000082C300008BA
:1002A000202A04DB203A00FA02F100207047914036
:1002B000C2F1200320FA03F3194390407047202A2B
:1002C00004DB203A21FA02F00021704721FA02F300
:1002D000D040C2F12002914008431946704700BF48
:1002E000FEE72DE9F043ADF26C4D80460E46914697
:1002F0000DF2044000F08CFD002514E0701BB0F5F9
:10030000806F02D94FF4806700E0771BBAB208EB28
:10031000050101A802F0F4FC3A4601A90DF20440DF
:1003200000F088FD3D44B542E8D30DF2044000F0F2
:1003300007FD002408E019F804100DF25C40005D90
:10034000814200D002E0641C102CF4DB00BF102CB2
:1003500004DA00200DF26C4DBDE8F0830120F9E7CE
:100360002DE9F047ADF5006D06460F4615469A4655
:100370002DB94FF0FF300DF5006DBDE8F087701915
:10038000B0F5800F02D94FF0FF30F4E7A7F100601D
:100390002844B0F5003F02D96FF00100EBE7524668
:1003A00029463046FFF79DFF10B96FF00200E2E7E3
:1003B000002416E0281BB0F5806F02D94FF4806945
:1003C00002E0281B1FFA80F931194A460DF58060BA
:1003D00002F096FC38194A460DF5806102F0F0F8FB
:1003E0004C44AC42E6D3002427E0281BB0F5806FD4
:1003F00002D94FF4806902E0281B1FFA80F93119F5
:100400004A460DF5806002F07BFC38194A46694681
:1004100000F0E0FE4FF000080CE00DF5806010F8F1
:1004200008001DF80810884202D06FF00300A2E710
:1004300008F10108C845F0DB4C44AC42D5D300209C
:1004400099E77047704721B1026842F001020260EB
:1004500004E002684FF6FE731A4002607047000025
:1004600001684FF6FE721140016000210160416099
:100470008160C1604B49884208D14A4908394968BE
:1004800041F00F01474A083A51608AE0454914316A
:10049000884208D143490839496841F0F001414A8E
:1004A000083A51607DE03F492831884208D13D49F2
:1004B0000839496841F470613A4A083A516070E07D
:1004C00038493C31884208D136490839496841F4F5
:1004D0007041344A083A516063E0324950318842F1
:1004E00008D130490839496841F470212D4A083A49
:1004F000516056E02B496431884208D129490839B6
:10050000496841F47001274A083A516049E0254999
:100510007831884208D123490839496841F070612F
:10052000204A083A51603CE01F49884206D1011F29
:10053000096841F00F01021F116032E01A491431BD
:10054000884208D11849091F096841F0F001164A8C
:10055000121F116025E014492831884208D1124940
:10056000091F096841F470610F4A121F116018E0F9
:100570000D493C31884208D10B49091F096841F4F3
:100580007041094A121F11600BE00749503188423F
:1005900007D10549091F096841F47021024A121F59
:1005A0001160704708000240080402401AB1036855
:1005B0000B43036002E003688B430360704710B590
:1005C0000022026847F6F0739A430C6A8B68234353
:1005D0000C6923434C6923438C692343CC6923432F
:1005E0004C6A23438C6A23431A430260CB684360FE
:1005F0000B6883604B68C36010BD70474FF0E02309
:100600001A6900210CE008E04FF0E0231B699342D7
:1006100003D04FF0E0231A6900E0F5E700BF491C62
:100620008142F0DB704710B5024606E0002102E08F
:1006300000BF4B1CD9B22D29FADB1300A2F1010433
:10064000A2B2F3D110BD000030B5044604254FF42A
:10065000302000F06FF80546042D17D10C480069D2
:1006600040F002000A49086108464461006940F010
:10067000400008614FF4302000F05CF80546044863
:10068000006941F6FD71084001490861284630BD06
:100690000020024004200B49C96811F0010F01D06D
:1006A00001200EE00749C96811F0040F01D00220B3
:1006B00007E00449C96811F0100F01D0032000E0E1
:1006C00004207047002002400348006940F0800089
:1006D00001490861704700000020024070B50446DF
:1006E0000D460426F00200F025F80646042E11D12E
:1006F0000948006940F00100074908612580F002BF
:1007000000F018F806460448006941F6FE710840FA
:1007100001490861304670BD00200240024803498B
:100720004860034848607047230167450020024045
:10073000AB89EFCD00B502460423FFF7ABFF0346BC
:1007400003E0FFF7A7FF0346521E012B01D1002A49
:10075000F7D102B90523184600BD2DE9F041024644
:1007600000250026002000230024002791F803C064
:100770000CF00F0591F803C01CF0100F03D091F896
:1007800002C04CEA050591F800C0BCF1000F31D061
:10079000146800202BE04FF0010C0CFA00F3B1F8C4
:1007A00000C00CEA03069E4220D183004FF00F0CDC
:1007B0000CFA03F7BC4305FA03FC4CEA040491F875
:1007C00003C0BCF1280F06D14FF0010C0CFA00FC5D
:1007D000C2F814C00AE091F803C0BCF1480F05D17B
:1007E0004FF0010C0CFA00FCC2F810C0401C0828A5
:1007F000D1D31460B1F800C0BCF1FF0F34DD5468F0
:1008000000202EE000F1080C4FF0010808FA0CF36C
:10081000B1F800C00CEA03069E4221D183004FF0DC
:100820000F0C0CFA03F7BC4305FA03FC4CEA040472
:1008300091F803C0BCF1280F05D100F1080C08FAAB
:100840000CF8C2F8148091F803C0BCF1480F07D12E
:1008500000F1080C4FF0010808FA0CF8C2F81080FB
:10086000401C0828CED35460BDE8F0814161704738
:10087000016170473EB55824684600F00FF8002526
:1008800003E01DF8050044406D1C0C2DF9DB04B994
:100890005824FF2C00D1852420463EBD0021064A65
:1008A00000BF05E013780370401C521C4B1CD9B2EA
:1008B0000C29F7DB70470000E8F7FF1F0948C088E4
:1008C0000849898808430749498808430549098830
:1008D0000843054908800846018804A001F0A2FEEB
:1008E00000BFFEE700000020100000200D0A5B485A
:1008F00046483D253034785D0D0A00002DE9F0436F
:10090000ADF2744D074688464FF000090DF20C40D9
:1009100000F07EFA0025002417E02C49601800F052
:10092000E4FC064628466D1C03A90E54320A2846EC
:100930006D1C0A54B5F5806F06D14FF480620DF23C
:100940000C4000F077FA0025A41CBC42E5D32DB181
:100950002A4603A90DF20C4000F06CFA0DF20C408F
:1009600000F0EEF93A461AA103A801F06BFE00244C
:100970000BE00DF26440025D1AA101A801F062FED5
:1009800001A903A8FFF718FC641C102CF1DB17A1C8
:1009900003A8FFF711FC03A800F098F9002408E071
:1009A00018F804100DF26440005D814200D002E0AE
:1009B000641C102CF4DB00BF102C04DA00200DF2B4
:1009C000744DBDE8F0830120F9E700000040000805
:1009D00046696C6553697A653D256420204D443530
:1009E0003D00000025303258000000000D0A0000D4
:1009F00070B504460D46074884420AD14FF4806220
:100A00002946054800F06CFA06463146024801F0D6
:100A1000F1FC70BD504354414309002070B50446B9
:100A20000548844207D1054800F092FA0546294658
:100A3000024801F0DFFC70BD5043544143090020DF
:100A40002DE9F04FA1B08046444620687B4988429A
:100A500004D04FF0FF3021B0BDE8F08F207980281E
:100A600002D06FF00100F6E77548D0F81D2075A19F
:100A70001DA801F0E7FDA11D1DA8FFF7A9FB10B1FE
:100A80006FF00200E7E794F805A0208B0190BAF11F
:100A9000000F28D10198142802D06FF00300DAE784
:100AA000C34610220BF11A016748FFF761FBD846D5
:100AB000DBF82A00654908600846006810B96FF045
:100AC0000400C8E700206249086062490860624982
:100AD0000860252000F0E0FA20685D490968FFF70A
:100AE00087FF0120B7E7BAF1020F7DD14746002604
:100AF00008E05548815D07F11A00805D814200D011
:100B000002E0761C102EF4DB00BF102E08DA53A092
:100B100000F0DCF82068FFF781FF6FF005009AE72E
:100B2000D7F82E50D7F82A000290022D0CD348494E
:100B300002980968884207D1454800682918434847
:100B40000068801C814208D949A000F0BFF82068E5
:100B5000FFF764FF6FF006007DE7AD1E2A4607F140
:100B60003201002001F0C6FF814607F13200691C06
:100B7000405C00021C9007F13200405D1C99084463
:100B800080B21C901C9949450AD041A000F09EF803
:100B900020682F490968FFF72BFF6FF007005AE71D
:100BA0002068264988420DD1002609E007F132006D
:100BB000805D2349097F484007F132018855761C42
:100BC000AE42F3D307F1320229462148006800F013
:100BD000A1F82148006828441F4908601C480068A3
:100BE00028441B49086000E026E01B4800681749BC
:100BF0000968884210DB144914480068FFF77EFE3C
:100C000040B929A000F062F82068FFF707FF6FF0F5
:100C1000080020E700201EE70D4829A1026803A86C
:100C200001F010FD03A800F051F820680849096898
:100C3000FFF7DEFE02200EE700BF0CE750435441F1
:100C400090000020256C75008000002034000020FA
:100C50003C00002040000020380000204D4435209A
:100C60004D6F64696679215265444F210D0A000079
:100C70004C656E677468206F72204F66667365748A
:100C8000206572726F72215265444F210D0A000077
:100C9000436865636B20435243206572726F722113
:100CA0005265444F210D0A00436865636B204D4433
:100CB00035206572726F72215265444F210D0A0012
:100CC0004842443D25640D0A0000000070B5054609
:100CD0002C460A20FFF792FC0BA001F0A3FC0BE0CE
:100CE00021780B4801F04AFA00BF4021084801F082
:100CF0007DF90028F9D0641C20780028F0D10A2062
:100D0000FFF77CFC70BD00005B4941505D000000B6
:100D1000003801402DE9F04104460D4616460027F3
:100D200014F0010F02D00020BDE8F081AAB20349FF
:100D30006018314601F044FC0120F5E7004000084E
:100D40002DE9F04190B0044620680E9060680F9045
:100D50002088C0F3C507382F02DAC7F1380001E058
:100D6000C7F17800804642462849204600F062F8E4
:100D70000026002518E004F11800E91C405C02067A
:100D800004F11800A91C405C42EA004204F118007A
:100D9000691C405C42EA002004F11801495D0843E7
:100DA0004DF82600761C2D1D0E2EE4D3694604F165
:100DB000080000F0E7FC0026002521E004F108000F
:100DC00010F8261050304155503830F82600C0F346
:100DD000072204F15800691C4254503850F826008C
:100DE000C0F3074204F15800A91C4254503850F88F
:100DF0002600000E04F15801EA1C8854761C2D1DB3
:100E0000042EDBD310B0BDE8F0810000CC2D00082B
:100E100000214160016005498160054AC260CA4302
:100E20000261034AD24342617047000001234567D3
:100E300089ABCDEF2DE9F04391B004460F4615463E
:100E40002088C0F3C509206800EBC50021688842EE
:100E500002D26068401C6060206800EBC500206022
:100E6000606800EB5570606033E017F8012B48466E
:100E700009F1010904F118010A54B9F1400F28D110
:100E80004FF0000800261AE004F11800F11C405C45
:100E9000020604F11800B11C405C42EA004204F171
:100EA0001800711C405C42EA002004F11801895DC1
:100EB000084301A941F8280008F10108361DB8F1DE
:100EC000100FE1D301A904F1080000F05BFC4FF022
:100ED00000092800A5F10105C7D111B0BDE8F083D4
:100EE0002DE9F04104460E46174625463221284694
:100EF000FFF757F911482860802028710220687197
:100F00000F48D0F81D200FA1A81D01F09BFB0E4833
:100F10000088401C80B20C490880E8821820288391
:100F200010220A4905F11A00FFF722F9C5F82A60D4
:100F3000C5F82E703220BDE8F081000050435441C6
:100F400090000020256C75003000002080000020FB
:100F500070B5044625462C212846FFF722F9104893
:100F6000286080202871002068710E48D0F81D206C
:100F70000DA1A81D01F066FB0A48007FE88212203F
:100F800028830849213105F11A00FFF73CF905488B
:100F9000B0F82F0068850020044908802C2070BD1F
:100FA0005043544190000020256C75003000002013
:100FB00000BFFEE7002003E00021074A1154401C57
:100FC000B0F5805FF8DB0021044A1180044A1180EB
:100FD000044A118070470000A80D00204C0000203A
:100FE0004E000020500000200022028082804280BB
:100FF000002108E00023821D02EB81025380821D44
:1010000022F82130491C0A29F4DB704770470000A0
:1010100070B5002100230F22C4780CB3164C24684D
:1010200004F4E064C4F5E064210AC1F10403CA4099
:10103000447804FA03F184781440214309010F4CE9
:101040000678A155047804F01F050124AC4005780A
:101050006D114FF0E02606EB8505C5F8004109E06B
:10106000047804F01F050124AC40054D0678761184
:1010700045F8264070BD00000CED00E000E400E003
:1010800080E100E002490143024A1160704700001C
:101090000000FA050CED00E004490978044A1170DB
:1010A000024908700121034A517170472B0000204A
:1010B0002C0000202400002029B1064A5269024376
:1010C000044B5A6104E0034A52698243014B5A615E
:1010D000704700000010024029B1064A926902439D
:1010E000044B9A6104E0034A92698243014B9A617E
:1010F000704700000010024030B50021002200249B
:1011000000232D4D6D6805F00C0121B1042905D097
:10111000082923D105E0294D056022E0284D05600E
:101120001FE0254D6D6805F47012234D6D6805F4C0
:101130008034022505EB92421CB9224D55430560CF
:101140000BE01D4D6D6815F4003F03D01E4D554357
:10115000056002E01A4D5543056002E0174D056039
:1011600000BF00BF144D6D6805F0F0010909174D6F
:101170006B5C0568DD4045600F4D6D6805F4E0610E
:10118000090A124D6B5C4568DD4085600A4D6D684B
:1011900005F46051C90A0D4D6B5C4568DD40C560C2
:1011A000054D6D6805F44041890B094D6B5CC568C0
:1011B000B5FBF3F5056130BD0010024000127A0066
:1011C000001BB70000093D00808D5B00540000202B
:1011D00064000020F0B505460B46164600270024A3
:1011E0000DE0281900F081F8024638467F1C1A5499
:1011F0004FEA122C38467F1C03F800C0A41CB442EE
:10120000EFDBF0BD10B5FFF735FB04463122024994
:101210000248FFF7DFFF10BD90000020003C0008EF
:1012200021B1028842F04002028004E002884FF6B9
:10123000BF731A40028070470246002013890B4298
:1012400001D0012000E000207047014688897047E6
:101250008181704710B50022028802F441520B8848
:101260004C8823438C882343CC8823430C89234315
:101270004C8923438C892343CC8923431A4302801E
:10128000838B4FF2FF74234083830B8A038210BD4C
:1012900010B5044600BF02210A48FFF7CDFF002821
:1012A000F9D021460748FFF7D3FF00BF01210548C9
:1012B000FFF7C2FF0028F9D00248FFF7C6FFC0B20F
:1012C00010BD00000030014030B503460C46154605
:1012D000002207E0184600F008F824F812009B1CD2
:1012E000501C82B2AA42F5DB30BD01460888704727
:1012F000704710B500F002F810BD00000CB50020DA
:10130000019000903048006840F480302E49086019
:1013100000BF2D48006800F4003000900198401C88
:101320000190009818B90198B0F5A06FF1D1264846
:10133000006810F4003F02D00120009001E000207E
:101340000090009801283ED12048006840F010002D
:101350001E4908600846006820F00300086008463F
:1013600000680860184840681749486008464068A7
:1013700048600846406848600846406820F47C1091
:1013800048600846406840F43020486008460068DD
:1013900040F08070086000BF0B48006810F0007FCC
:1013A000FAD00948406820F0030007494860084621
:1013B000406840F00200486000BF0348406800F009
:1013C0000C000828F9D10CBD00100240002002409A
:1013D00030B502460B461946144607E008782578D2
:1013E000A84201D0012030BD491C641C08780028A7
:1013F000F4D100BFF7E7000010B588B000203749EE
:1014000008603749086037480078362802D05828E5
:1014100061D149E034A0FFF759FC00243BE037A03C
:10142000FFF754FC3C498A6948690B1D3B49FEF7AC
:1014300097FF001D052820D2DFE800F01A15100BD9
:10144000030037A0FFF742FC5820FFF725FE08B045
:1014500010BD38A1684601F0F5F813E038A16846E0
:1014600001F0F0F80EE039A1684601F0EBF809E070
:1014700038A1684601F0E6F804E039A1684601F0B9
:10148000E1F800BF00BF2AA16846FEF795FE684656
:10149000FFF71CFC641C032CC1DB34A0FFF716FC17
:1014A0005820FFF7F9FD16E031221B493548FFF7B8
:1014B00091FE0422184934A0FEF798FE40B1164868
:1014C00031A109680160312201462E4801F026F859
:1014D00001F040FB00BF00BF00BFB8E718000020CC
:1014E000140000202B0000204558464C4153485F13
:1014F000555044415445210D0A000000436F707956
:1015000020417070206461746120546F204D6375B8
:101510002E2E2E0D0A000000900000200040000832
:10152000436F7079417070546F4D6375204F4B213C
:101530000D0A0000457874416464724572720000BF
:10154000496E744164647245727200004D643545A1
:1015500072720000556E4D6174636844617461007D
:101560004F7468657245727200000000436F7079B5
:10157000417070546F4D6375204661696C21212163
:101580000D0A0000003C000846544F4B00000000CC
:1015900010B501201549C87015480068401C144951
:1015A0000860322804DB0020086001200F49087120
:1015B00010480078012817D10F480068401C0E49D8
:1015C000086008460068B0F5FA7F0DDD0B480CA1F5
:1015D00009680160042201460B4800F09FFF0BA040
:1015E00001F020F800BFFEE710BD0000240000203D
:1015F00008000020530000200C0000209000002074
:1016000046544F4B00000000003C0008777269749C
:1016100065204578466C617368206572726F72212F
:101620000D0A7265626F6F74204D435520616E64C0
:1016300020476F746F20415050210D0A00000000B8
:1016400010B51348006840F00100114908600846D1
:101650004068104908400E494860084600680E4935
:1016600008400B4908600846006820F480200860A4
:101670000846406820F4FE0048604FF41F00886070
:10168000FFF737FE4FF000600449086010BD00000E
:10169000001002400000FFF8FFFFF6FE08ED00E03A
:1016A00010B52B480068401C04D029480068401C35
:1016B0002749086027480078122817D12448006875
:1016C000042800D210BD312223492448FFF782FDAF
:1016D0000422214922A0FEF789FD18B93620FFF720
:1016E000DBFC33E05820FFF7D7FC2FE019480078E7
:1016F000252816D11C480068401C1B490860022898
:1017000024DD0020086019480068012803D017482C
:10171000006802281AD1164801681648FFF768F9D0
:1017200014E00C480078362810D00A480078582871
:101730000CD107480068042800D2C3E704480078A9
:1017400010F0010F02D00CA0FFF7C0FA00BFB9E7FC
:10175000180000202B00002090000020003C000812
:10176000466F5461000000001C0000202000002093
:101770003C000020504354414E6F20417070210DB9
:101780000A000000F0B505460C4628686968AA689A
:10179000EB6801EA020623EA01073E4327683E445C
:1017A000FE4F3E443044C60146EA5060084400EA19
:1017B000010622EA00073E4367683E44F84F3E4474
:1017C00033441E0346EA1353034403EA000621EAA6
:1017D00003073E43A7683E44F24F3E44324456045A
:1017E00046EAD2321A4402EA030620EA02073E43DE
:1017F000E7683E44EC4F3E4431448E0546EA912171
:10180000114401EA020623EA01073E4327693E44E8
:10181000E64F3E443044C60146EA5060084400EAC0
:10182000010622EA00073E4367693E44E04F3E441A
:1018300033441E0346EA1353034403EA000621EA35
:1018400003073E43A7693E44DA4F3E443244560400
:1018500046EAD2321A4402EA030620EA02073E436D
:10186000E7693E44D44F3E4431448E0546EA912117
:10187000114401EA020623EA01073E43276A3E4477
:10188000CE4F3E443044C60146EA5060084400EA68
:10189000010622EA00073E43676A3E44C84F3E44C1
:1018A00033441E0346EA1353034403EA000621EAC5
:1018B00003073E43A76A3E44A6F524464F3E324402
:1018C000560446EAD2321A4402EA030620EA020724
:1018D0003E43E76A3E44BB4F3E4431448E0546EAF0
:1018E0009121114401EA020623EA01073E43276BD6
:1018F0003E44B54F3E443044C60146EA5060084479
:1019000000EA010622EA00073E43676B3E44AF4F00
:101910003E4433441E0346EA1353034403EA0006DD
:1019200021EA03073E43A76B3E44A94F3E4432449D
:10193000560446EAD2321A4402EA030620EA0207B3
:101940003E43E76B3E44A34F3E4431448E0546EA96
:101950009121114401EA030622EA03073E43676826
:101960003E449D4F3E443044460146EAD060084420
:1019700000EA020621EA02073E43A7693E44974F68
:101980003E4433445E0246EAD353034403EA01066D
:1019900020EA01073E43E76A3E44914F3E44324409
:1019A000960346EA92421A4402EA000623EA000736
:1019B0003E4327683E448B4F3E4431440E0546EA81
:1019C0001131114401EA030622EA03073E43676925
:1019D0003E44854F3E443044460146EAD0600844C8
:1019E00000EA020621EA02073E43A76A3E447F4F0F
:1019F0003E4433445E0246EAD353034403EA0106FD
:101A000020EA01073E43E76B3E44794F3E443244AF
:101A1000960346EA92421A4402EA000623EA0007C5
:101A20003E4327693E44734F3E4431440E0546EA27
:101A30001131114401EA030622EA03073E43676AB3
:101A40003E446D4F3E443044460146EAD06008446F
:101A500000EA020621EA02073E43A76B3E44674FB5
:101A60003E4433445E0246EAD353034403EA01068C
:101A700020EA01073E43E7683E44614F3E4432445A
:101A8000960346EA92421A4402EA000623EA000755
:101A90003E43276A3E445B4F3E4431440E0546EACE
:101AA0001131114401EA030622EA03073E43676B42
:101AB0003E44554F3E443044460146EAD060084417
:101AC00000EA020621EA02073E43A7683E444F4F60
:101AD0003E4433445E0246EAD353034403EA01061C
:101AE00020EA01073E43E7693E44494F3E44324401
:101AF000960346EA92421A4402EA000623EA0007E5
:101B00003E43276B3E44434F3E4431440E0546EA74
:101B10001131114481EA02065E4067693E443E4F3E
:101B20003E443044060146EA1070084480EA01064B
:101B30005640276A3E44394F3E443344DE0246EA6B
:101B40005353034483EA00064E40E76A3E44344F51
:101B50003E443244160446EA12421A4482EA03061C
:101B60004640A76B3E442F4F3E443144CE0546EAE3
:101B70005121114481EA02065E4067683E442A4FC3
:101B80003E443044060146EA1070084480EA0106EB
:101B9000564027693E44254F3E4449E078A46AD721
:101BA00056B7C7E8DB702024EECEBDC1AF0F7CF581
:101BB0002AC68747134630A8019546FDD898806904
:101BC000AFF7448BBED75C892211906B937198FD5F
:101BD0008E4379A62108B44962251EF640B340C061
:101BE000515A5E26AAC7B6E95D102FD65314440297
:101BF00081E6A1D8C8FBD3E7E6CDE121D60737C3FC
:101C0000870DD5F4ED145A4505E9E3A9F8A3EFFCD7
:101C1000D9026F678A4C2A8D4239FAFF81F67187A3
:101C200022619D6D0C38E5FD44EABEA4A9CFDE4BD0
:101C30003344DE0246EA5353034483EA00064E402F
:101C4000E7693E449F4F3E443244160446EA12423E
:101C50001A4482EA03064640A76A3E449A4F3E442D
:101C60003144CE0546EA5121114481EA02065E4024
:101C7000676B3E44954F3E443044060146EA10707F
:101C8000084480EA0106564027683E44904F3E448F
:101C90003344DE0246EA5353034483EA00064E40CF
:101CA000E7683E448B4F3E443244160446EA1242F3
:101CB0001A4482EA03064640A7693E44864F3E44E2
:101CC0003144CE0546EA5121114481EA02065E40C4
:101CD000676A3E44814F3E443044060146EA107034
:101CE000084480EA01065640276B3E447C4F3E4440
:101CF0003344DE0246EA5353034483EA00064E406F
:101D0000E76B3E44774F3E443244160446EA1242A3
:101D10001A4482EA03064640A7683E44724F3E4496
:101D20003144CE0546EA5121114461EA030656408A
:101D300027683E446D4F3E443044860146EA906039
:101D4000084460EA02064E40E7693E44684F3E445C
:101D500033449E0246EA9353034463EA0106464035
:101D6000A76B3E44634F3E443244D60346EA524298
:101D70001A4462EA00065E4067693E445E4F3E4494
:101D800031444E0546EAD121114461EA030656402A
:101D9000276B3E44594F3E443044860146EA9060EA
:101DA000084460EA02064E40E7683E44544F3E4411
:101DB00033449E0246EA9353034463EA01064640D5
:101DC000A76A3E444F4F3E443244D60346EA52424D
:101DD0001A4462EA00065E4067683E444A4F3E4449
:101DE00031444E0546EAD121114461EA03065640CA
:101DF000276A3E44454F3E443044860146EA90609F
:101E0000084460EA02064E40E76B3E44404F3E44C1
:101E100033449E0246EA9353034463EA0106464074
:101E2000A7693E443B4F3E443244D60346EA524201
:101E30001A4462EA00065E40676B3E44364F3E44F9
:101E400031444E0546EAD121114461EA0306564069
:101E500027693E44314F3E443044860146EA906053
:101E6000084460EA02064E40E76A3E442C4F3E4476
:101E700033449E0246EA9353034463EA0106464014
:101E8000A7683E44274F3E443244D60346EA5242B6
:101E90001A4462EA00065E40676A3E44224F3E44AE
:101EA00031444E0546EAD12111442E6806442E6085
:101EB0006E680E446E60AE681644AE60EE681E44F6
:101EC000EE60F0BD604BBBF670BCBFBEC67E9B280B
:101ED000FA27A1EA8530EFD4051D880439D0D4D97A
:101EE000E599DBE6F87CA21F6556ACC4442229F4D0
:101EF00097FF2A43A72394AB39A093FCC3595B6592
:101F000092CC0C8F7DF4EFFFD15D84854F7EA86F5E
:101F1000E0E62CFE144301A3A111084E827E53F784
:101F200035F23ABDBBD2D72A91D386EB08B540F241
:101F30002441174800F067F840B315480088009026
:101F40001348001D008800901248C06D40F23441D3
:101F5000081A009000210F485830FEF774FA0E4816
:101F6000007850B90D490E48009AFEF701F90D4965
:101F70000098088001200849087040F23440054963
:101F8000C865012103485830FEF75DFA08BD00001E
:101F90000038014000000240240000200F0500200E
:101FA000DB0000204400002010B5FFF7BFFF10BD8C
:101FB00001F40072B2F5007F00D100BFCA43028075
:101FC000704721B1828942F40052828104E0828903
:101FD0004DF6FF731A40828170471AB1838A0B4312
:101FE000838202E0838A8B4383827047024600200B
:101FF000B1F5007F00D100BF13880B4201D0012052
:1020000000E00020704770B5024600240023002540
:102010000020A1F510666A3E00D100BFC1F3421551
:1020200001F01F03012606FA03F3012D02D1968960
:10203000334006E0022D02D1168A334001E0968A31
:1020400033400C12012606FA04F41688344013B10A
:102050000CB1012000E0002070BDF0B50346002463
:10206000002600250020A1F510676A3F00D100BFBF
:102070001846C1F3421401F01F06012707FA06F5BE
:10208000012C01D10C3004E0022C01D1103000E011
:1020900014301AB107682F43076002E00768AF43A6
:1020A0000760F0BD2DE9F04786B005460E460024D6
:1020B000A24600BFA1460027B08900B100BF2F464D
:1020C0002C8A4CF6FF700440F08804432C82AC89C3
:1020D0004EF6F3100440B0883189084371890843F3
:1020E0000443AC81AC8A4FF6FF400440B0890443FE
:1020F000AC8201A8FFF700F81F48874202D1DDF843
:1021000010A001E0DDF80CA0A88910F4004F08D061
:102110000AEBCA0000EB0A1031684900B0FBF1F885
:1021200007E00AEBCA0000EB0A1031688900B0FB37
:10213000F1F86420B8FBF0F004012009642101FBF0
:102140001089A88910F4004F08D0322000EBC90094
:10215000B0FBF1F000F00700044308E0322000EB90
:1021600009106421B0FBF1F000F00F0004432C8152
:1021700006B0BDE8F087000000380140C1F3080256
:102180008280704700B58DB001210846FEF794FFAC
:102190002B48FEF765F92B4801902B480290102040
:1021A0000390642004900020059080200690002079
:1021B0000790089009900A900B9001A92048FEF71B
:1021C000FEF90E208DF8300003208DF8310002203A
:1021D0008DF8320001208DF833000CA8FEF718FFAF
:1021E000012202211648FEF7E1F900211448FEF70A
:1021F0002AF913481430FEF733F9124801901348B6
:1022000002900020039040F234400490002005909A
:102210008020069000200790089009904FF400500D
:102220000A9000200B9001A905481430FEF7C7F969
:10223000012103481430FEF706F90DB000BD00007F
:102240004400024004380140430900200F050020EB
:1022500000B587B0012144F20400FEF73DFF4FF4C2
:102260000070ADF8140018208DF8170003208DF8C9
:10227000160005A92E48FEF770FA4FF48060ADF8FD
:10228000140004208DF8170003208DF8160005A90E
:102290002748FEF762FA4FF4E13001900020ADF8D4
:1022A0000800ADF80A00ADF80C00ADF810000C20E5
:1022B000ADF80E0001A91F48FFF7F4FE01211D48EB
:1022C000FFF77FFE4FF4E060FEF7DCFE25208DF87F
:1022D000180000208DF819008DF81A0001208DF8E3
:1022E0001B0006A8FEF794FE40211248FFF760FE8F
:1022F000002240F227710F48FFF7AFFE002240F2A4
:1023000025510C48FFF7A9FE012240F2244109485B
:10231000FFF7A3FE012240210648FFF75EFE0022E0
:1023200080210448FFF759FEFFF72CFF07B000BDDE
:10233000000801400038014010B51A480078122802
:102340000ED119A11C48FFF743F848B91BA0FEF7AE
:10235000BDFC1E48FEF762FB1BA0FEF7B7FC10BDDC
:102360001B4801881448FEF76BFB044634B919A0DA
:10237000FEF7ACFC5820FEF78FFEF0E714F1020FD9
:1023800008DA14F1060F05DD15A0FEF79FFC5820B2
:10239000FEF782FE0020154908601548046000BF62
:1023A000DDE700002B000020444F574E4C4F4144C6
:1023B0005F41505000000000DB000020444F574EAA
:1023C0004C4F41445F4150500D0A0000504354416E
:1023D00044000020436F6D706C65746564210000DB
:1023E0004941502053746F70210D0A001C000020D9
:1023F0002000002070B505460E4600240BE0295D44
:102400000648FFF7BBFE00BF40210448FFF7EEFD82
:102410000028F9D0641CB442F1DB70BD00380140E3
:1024200000BFFEE710B586B000F038F8102119485B
:10243000FEF71EFA0020ADF804004FF48270ADF8EC
:1024400006000020ADF808000220ADF80A000120C7
:10245000ADF80C004002ADF80E000820ADF81000F9
:102460000020ADF812000720ADF8140001A90A48B9
:10247000FEF7F0FE01210848FEF7D2FE4FF47A7015
:10248000FEF7D1F800F092FC00F068FC0446012051
:1024900006B010BD000801400030014008B5012120
:1024A0000420FEF719FE01210803FEF715FE202087
:1024B000ADF8000003208DF8020018208DF803000D
:1024C00069461448FEF749F98020ADF800006946D6
:1024D0001048FEF742F94020ADF8000004208DF8C6
:1024E000030069460B48FEF738F91020ADF80000EC
:1024F0008DF8030069460748FEF72FF90120ADF873
:10250000000010208DF8030069460348FEF725F906
:1025100008BD000000080140000C01402DE9F05FFB
:1025200005460E461746B5F1006F02D32248854294
:1025300002D3A346BDE8F09FA805800D00D0F9E7BF
:102540004FF400721D492846FEF7BEFE002411E03C
:102550004FF6FF7000EA440816F8081008F1010071
:10256000305C01EB00201FFA80FA144820F814A018
:10257000601C84B207EBD771B4EB610FE8DBFEF7A8
:10258000CDF82846FEF760F88146B9F1040F00D077
:10259000D0E7002408E0094A32F8141005EB4400A3
:1025A000FEF79CF8601C84B2B4F5007FF3DBFEF705
:1025B0008BF800BFBEE7000000000208A809002059
:1025C0002DE9F04705460E469046B5F1006F02D35F
:1025D0001348854201D3BDE8F087A805800D00D0DF
:1025E000F9E7FEF79BF82846FEF72EF80746042F7A
:1025F00000D0F0E700240CE0315D601C305C01EBA2
:1026000000201FFA80F928194946FEF767F8A01C38
:1026100084B24445F0DBFEF757F800BFDBE700006B
:10262000000002080FB4054B10B503A9044A029834
:1026300000F02CF810BC5DF814FB0000312B0008F2
:102640007C0000200FB4084B10B504A902AA03981F
:1026500000F01CF8044602A9002000F046FA2046CB
:1026600010BC5DF814FB0000EB2A000802E008C86B
:10267000121F08C1002AFAD170477047002001E0FC
:1026800001C1121F002AFBD1704700002DE9FF4F46
:102690008DB00F4605460026DEE1252874D10024C2
:1026A0006D1CF149A246A14601222B78203B02FA7B
:1026B00003F0084202D004436D1CF6E728782A286C
:1026C00010D06FF02F022878A0F13001092915D819
:1026D0000AEB8A0102EB410144F0020400EB010A1B
:1026E0006D1CF0E757F804ABBAF1000F03DA44F4BD
:1026F0000054CAF1000A44F002046D1C28782E2808
:1027000017D115F8010F44F004042A280ED06FF0F9
:102710002F022878A0F1300109290AD809EB890194
:1027200002EB410100EB01096D1CF2E757F8049B35
:102730006D1C28786C280FD006DC4C2817D0682830
:102740000DD06A2814D104E0742810D07A280FD153
:102750000DE044F400140AE044F4801401E044F471
:1027600040146978814202D16D1C04F580146D1CFF
:102770002A786E2A20D00DDC632A33D005DC002AAB
:102780006FD0582A12D1A2E011E0642A6AD0692AD7
:102790000CD167E0732A2FD004DC6F2A6FD0702A27
:1027A00004D199E0752A6BD0782A6AD01046DDE909
:1027B0000F129047761C4EE1C4F30250022806D057
:1027C00003280AD0042801CF0AD0066043E101CFD4
:1027D0004FEAE671C0E900613DE101CF06803AE1D0
:1027E000067038E117F8040B8DF8000000208DF812
:1027F0000100EB46012003E057F804BB4FF0FF3027
:1028000061074FF0000102D40DE008F10101884694
:1028100049450FDA8045F8DB1BF808100029F4D190
:1028200008E008F1010188468142FADB1BF8081034
:102830000029F6D1DDE90F23AAEB080081462146E5
:1028400000F03BF9304400EB080604E0DDE90F122C
:102850001BF8010B9047B8F10108F7D22146484612
:10286000F4E0FDE00A21C4F302534FF0000B08919D
:10287000022B07D001CFC117032B09D00AE034E0A7
:1028800023E024E0FF1D27F00707F7E8020105E039
:1028900000B2C117042B01D140B2C117002907DAD9
:1028A0004FF0000CD0EB0C006CEB01012D2302E08B
:1028B000230504D52B238DF82430012303E0E307FF
:1028C00001D02023F7E7984650E00A210EE01020BF
:1028D0004FF0000B08900CE010214FF0000B44F07B
:1028E00004044FF00809089103E008214FF0000BA1
:1028F0000891C4F30253022B04D001CF0021032B13
:1029000006D006E0FF1D27F00707F7E8020103E005
:1029100080B2042B00D1C0B24FF00008230725D5A8
:10292000702A2AD0DDF820C08CF0100C5CEA0B0C69
:1029300009D150EA010306D030238DF824308DF8F8
:10294000252002239846DDF820C08CF0080C5CEAB4
:102950000B0C0BD150EA010301D1630706D53023DC
:102960008DF824304FF00108A9F10109582A09D047
:102970003EA20B9208AA0A9211E040238DF824305F
:102980000123DFE73EA2F4E75B46089AFDF744FC2B
:102990000B9B9B5C0A9AA2F101020A92137050EA07
:1029A0000102F1D10A98ADEB000000F1200B6007A5
:1029B00002D524F4803401E04FF00109D94502DD4D
:1029C000A9EB0B0000E0002000EB0B014144089054
:1029D000AAEB010AE00306D4DDE90F2321465046A5
:1029E00000F06BF80644002008E009A911F809007E
:1029F000DDE90F129047761C09F101008146404540
:102A0000F3DBE0030CD5DDE90F232146504600F04F
:102A100054F8064404E0DDE90F1230209047761C9C
:102A20000899481E08900029F5DC08E00A980A99E0
:102A30000078491C0A91DDE90F129047761CBBF122
:102A40000001ABF1010BF1DC21465046DDE90F231B
:102A500000F020F806446D1C287800287FF41DAE95
:102A600011B03046BDE8F08F092801003031323313
:102A700034353637383961626364656600000000BA
:102A800030313233343536373839414243444546A4
:102A9000000000002DE9F041044600251E461746BF
:102AA000880405D406E039462020B04705F1010529
:102AB000641EF8D52846BDE8F0812DE9F0410446B2
:102AC00000251E469046C80301D5302700E0202788
:102AD000880405D506E041463846B04705F10105B2
:102AE000641EF8D52846BDE8F0810A68531C0B60C7
:102AF00010707047F0B507460C461546002606E0F4
:102B000014F8011B384600F007F80746761CAE4261
:102B1000F6D33846F0BD0000024682EA0100C0B29A
:102B2000024B33F8100080EA222070470C2E000878
:102B300070B504460D46E1B20548FFF71FFB00BF24
:102B400040210348FFF752FA0028F9D0204670BD13
:102B50000038014010B51B4800681B490840B0F11F
:102B6000005F2AD119A0FEF7B1F800204FF0E02154
:102B70000861002240F225511748FFF76EFA002243
:102B800040F224411448FFF768FA002240F227710E
:102B90001148FFF762FA002240210F48FFF71DFAA3
:102BA00000210E48FDF74FFC00210C481430FDF7C2
:102BB0004AFC044800F01AF802E009A0FEF786F883
:102BC00010BD0000004000080000FE2F476F546F4A
:102BD0004170700D0A0000000038014044000240BE
:102BE0004E6F20417070320D0A00000010B504468F
:102BF0006068044908602068FDF7A4FA014800688D
:102C0000804710BD48000020FFF70CFCFEF7D2F90A
:102C10003048FEF7E9F9FFF71BFB2F4800686422F4
:102C2000B0FBF2F1B1F1807F01D301201DE021F072
:102C30007F40401E4FF0E022506150170F220028C5
:102C400007DA13071D0E254B00F00F04241F1D5536
:102C500003E013071C0E224B1C5400BF00204FF052
:102C6000E022906107201061002008B100BFFEE75C
:102C70001CA0FEF72BF8FEF7C5FA1F4800210160E3
:102C8000818081711220FEF707FA22E01A4800784D
:102C900048B1FFF751FB00201749087040F234415A
:102CA0001648FDF77EFA1448407920B100201249F9
:102CB0004871FEF7A1FB1048C07810B100200E4902
:102CC000C8700D48007920B100200B490871FEF74B
:102CD000E7FCDBE7A81D00206800002018ED00E0FD
:102CE00000E400E04869676F734C2049415020566A
:102CF000322E300D0A00000024000020DB000020EE
:102D00002DE9F04105460C46174610211248FDF703
:102D1000ADFD0B20FEF7BCFAC4F30740FEF7B8FA8E
:102D2000C4F30720FEF7B4FAE0B2FEF7B1FAFF20D1
:102D3000FEF7AEFA2870002605E0FF20FEF7A8FA9D
:102D4000A855701C86B2BE42F7DB10210248FDF781
:102D50008FFDBDE8F0810000000801402DE9F04141
:102D6000002400250026002710210F48FDF77EFDD6
:102D70009F20FEF78DFAFF20FEF78AFA0546FF2016
:102D8000FEF786FA0646FF20FEF782FA0746102174
:102D90000548FDF76DFD280440EA062040EA0704D7
:102DA0002046BDE8F08100000008014010B5102168
:102DB0000548FDF75BFD0620FEF76AFA1021024880
:102DC000FDF756FD10BD0000000801408000000026
:102DD00000000000000000000000000000000000F3
:102DE00000000000000000000000000000000000E3
:102DF00000000000000000000000000000000000D3
:102E00000000000000000000000000000000C1C041
:102E100081C1400101C3C003800241C201C6C00696
:102E2000800741C70005C1C581C4400401CCC00C66
:102E3000800D41CD000FC1CF81CE400E000AC1CA26
:102E400081CB400B01C9C009800841C801D8C01816
:102E5000801941D9001BC1DB81DA401A001EC1DE96
:102E600081DF401F01DDC01D801C41DC0014C1D486
:102E700081D5401501D7C017801641D601D2C012A6
:102E8000801341D30011C1D181D0401001F0C03076
:102E9000803141F10033C1F381F240320036C1F696
:102EA00081F7403701F5C035803441F4003CC1FC66
:102EB00081FD403D01FFC03F803E41FE01FAC03A26
:102EC000803B41FB0039C1F981F840380028C1E856
:102ED00081E9402901EBC02B802A41EA01EEC02E96
:102EE000802F41EF002DC1ED81EC402C01E4C02486
:102EF000802541E50027C1E781E640260022C1E2A6
:102F000081E3402301E1C021802041E001A0C060B5
:102F1000806141A10063C1A381A240620066C1A695
:102F200081A7406701A5C065806441A4006CC1AC65
:102F300081AD406D01AFC06F806E41AE01AAC06A25
:102F4000806B41AB0069C1A981A840680078C1B815
:102F500081B9407901BBC07B807A41BA01BEC07E95
:102F6000807F41BF007DC1BD81BC407C01B4C07485
:102F7000807541B50077C1B781B640760072C1B2A5
:102F800081B3407301B1C071807041B00050C190F5
:102F9000819140510193C053805241920196C05695
:102FA000805741970055C19581944054019CC05C65
:102FB000805D419D005FC19F819E405E005AC19A25
:102FC000819B405B0199C059805841980188C04855
:102FD00080494189004BC18B818A404A004EC18E95
:102FE000818F404F018DC04D804C418C0044C18485
:102FF000818540450187C047804641860182C042A5
:10300000804341830041C181818040402C300008D1
:1030100000000020800000006C260008AC30000892
:1030200080000020582100007C26000800000000DD
:103030000000000000000000000000000000000090
:103040000000000000000000000000000000000080
:103050000000000000000000000000000000000070
:103060000000000000000000000000000000000060
:103070000000000000000000000000000000000050
:10308000000000000102030401020304060708090E
:103090000204060800366E01000000000000000077
:0C30A000010203040607080900000000FC
:0400000508000131BD
:00000001FF
